 lcdad

 Timestamp is 4fb04cba (Mon May 14 12:07:22 2012)

 Preferred load address is 10000000

 Start         Length     Name                   Class
 0001:00000000 00000004H .CRT$XCA                CODE
 0001:00000004 00000004H .CRT$XCZ                CODE
 0001:00000008 00000004H .CRT$XIA                CODE
 0001:0000000c 00000004H .CRT$XIZ                CODE
 0001:00000010 00000004H .CRT$XPA                CODE
 0001:00000014 00000004H .CRT$XPZ                CODE
 0001:00000018 00000004H .CRT$XTA                CODE
 0001:0000001c 00000004H .CRT$XTZ                CODE
 0001:00000020 000002c8H .rdata                  CODE
 0001:000002e8 00000022H .rdata$debug            CODE
 0001:0000030c 00000d10H .text                   CODE
 0001:0000101c 00000014H .xdata                  CODE
 0001:00001030 00000028H .idata$2                CODE
 0001:00001058 00000014H .idata$3                CODE
 0001:0000106c 00000054H .idata$4                CODE
 0001:000010c0 0000006eH .idata$6                CODE
 0001:00001130 000000d8H .edata                  CODE
 0002:00000000 00000054H .idata$5                DATA
 0002:00000058 000004d4H .data                   DATA
 0002:00000530 00000014H .bss                    DATA
 0003:00000000 000000e8H .pdata                  DATA

  Address         Publics by Value              Rva+Base       Lib:Object

 0000:00000000       ___safe_se_handler_count   00000000     <absolute>
 0000:00000000       ___safe_se_handler_table   00000000     <absolute>
 0001:00000000       __xc_a                     10001000     corelib0:crt0init.obj
 0001:00000004       __xc_z                     10001004     corelib0:crt0init.obj
 0001:00000008       __xi_a                     10001008     corelib0:crt0init.obj
 0001:0000000c       __xi_z                     1000100c     corelib0:crt0init.obj
 0001:00000010       __xp_a                     10001010     corelib0:crt0init.obj
 0001:00000014       __xp_z                     10001014     corelib0:crt0init.obj
 0001:00000018       __xt_a                     10001018     corelib0:crt0init.obj
 0001:0000001c       __xt_z                     1000101c     corelib0:crt0init.obj
 0001:0000003c       ??_C@_19OBGHODPD@?$AAM?$AAo?$AAd?$AAe?$AA?$AA@ 1000103c     LCDAD.obj
 0001:000002dc       ??_C@_1M@LCEEOPDH@?$AAI?$AA2?$AAC?$AA1?$AA?3?$AA?$AA@ 100012dc     lcdeeprom.obj
 0001:0000030c       DllMain                    1000130c f   LCDAD.obj
 0001:00000324       ?Init@@YAPAXPAX@Z          10001324 f   LCDAD.obj
 0001:0000037c       ?Deinit@@YAHPAX@Z          1000137c f   LCDAD.obj
 0001:00000384       ?Open@@YAPAXPAXKK@Z        10001384 f   LCDAD.obj
 0001:0000038c       ?Close@@YAHPAX@Z           1000138c f   LCDAD.obj
 0001:00000394       ?Read@@YAKPAXPAEK@Z        10001394 f   LCDAD.obj
 0001:0000039c       ?Write@@YAKPAXPAEK@Z       1000139c f   LCDAD.obj
 0001:000003a4       ?Seek@@YAKPAXJK@Z          100013a4 f   LCDAD.obj
 0001:000003ac       ?IOControl@@YAHPAXKPAEK1KPAK@Z 100013ac f   LCDAD.obj
 0001:000003b4       ?PowerUp@@YAHPAX@Z         100013b4 f   LCDAD.obj
 0001:000003bc       ?PowerDown@@YAHPAX@Z       100013bc f   LCDAD.obj
 0001:000004c0       ?WriteI2CRegister@@YAHPAXEEE@Z 100014c0 f   lcdeeprom.obj
 0001:0000052c       ?WriteI2CRegister@@YAHPAXEGE@Z 1000152c f   lcdeeprom.obj
 0001:00000970       ?GetModeFromEEPROM@@YAPAULCD_MODE_INFO@@XZ 10001970 f   lcdeeprom.obj
 0001:00000bdc       DisableThreadLibraryCalls  10001bdc f   coredll:COREDLL.dll
 0001:00000bec       RegCloseKey                10001bec f   coredll:COREDLL.dll
 0001:00000bfc       RegSetValueExW             10001bfc f   coredll:COREDLL.dll
 0001:00000c0c       OpenDeviceKey              10001c0c f   coredll:COREDLL.dll
 0001:00000c1c       Sleep                      10001c1c f   coredll:COREDLL.dll
 0001:00000c2c       I2CTransfer                10001c2c f   i2csdk:I2CSDK.dll
 0001:00000c3c       I2CSetFrequency            10001c3c f   i2csdk:I2CSDK.dll
 0001:00000c4c       I2CSetMasterMode           10001c4c f   i2csdk:I2CSDK.dll
 0001:00000c5c       I2COpenHandle              10001c5c f   i2csdk:I2CSDK.dll
 0001:00000c6c       I2CCloseHandle             10001c6c f   i2csdk:I2CSDK.dll
 0001:00000d80       _DllMainCRTStartup         10001d80 f   corelib0:pegdmain.obj
 0001:00000eac       _cexit                     10001eac f   corelib0:cexit.obj
 0001:00000ec8       _initterm                  10001ec8 f   corelib0:crt0dat.obj
 0001:00000efc       _cinit                     10001efc f   corelib0:crt0dat.obj
 0001:00000f30       __security_init_cookie     10001f30 f   corelib0:seccinit.obj
 0001:00000f8c       memcmp                     10001f8c f   corelib1:COREDLL.dll
 0001:00000f9c       memcpy                     10001f9c f   corelib1:COREDLL.dll
 0001:00000fac       _XcptFilter                10001fac f   corelib1:COREDLL.dll
 0001:00000fbc       __C_specific_handler       10001fbc f   corelib1:COREDLL.dll
 0001:00000fcc       free                       10001fcc f   corelib1:COREDLL.dll
 0001:00000fdc       __security_gen_cookie2     10001fdc f   corelib1:COREDLL.dll
 0001:00000fec       DeleteCriticalSection      10001fec f   coredll:COREDLL.dll
 0001:00000ffc       InterlockedExchange        10001ffc f   coredll:COREDLL.dll
 0001:0000100c       TerminateProcess           1000200c f   coredll:COREDLL.dll
 0001:00001030       __IMPORT_DESCRIPTOR_COREDLL 10002030     coredll:COREDLL.dll
 0001:00001044       __IMPORT_DESCRIPTOR_I2CSDK 10002044     i2csdk:I2CSDK.dll
 0001:00001058       __NULL_IMPORT_DESCRIPTOR   10002058     coredll:COREDLL.dll
 0002:00000000       __imp_DisableThreadLibraryCalls 10003000     coredll:COREDLL.dll
 0002:00000004       __imp_RegCloseKey          10003004     coredll:COREDLL.dll
 0002:00000008       __imp_RegSetValueExW       10003008     coredll:COREDLL.dll
 0002:0000000c       __imp_OpenDeviceKey        1000300c     coredll:COREDLL.dll
 0002:00000010       __imp_Sleep                10003010     coredll:COREDLL.dll
 0002:00000014       __imp_TerminateProcess     10003014     coredll:COREDLL.dll
 0002:00000018       __imp_InterlockedExchange  10003018     coredll:COREDLL.dll
 0002:0000001c       __imp_DeleteCriticalSection 1000301c     coredll:COREDLL.dll
 0002:00000020       __imp_memcmp               10003020     corelib1:COREDLL.dll
 0002:00000024       __imp_memcpy               10003024     corelib1:COREDLL.dll
 0002:00000028       __imp__XcptFilter          10003028     corelib1:COREDLL.dll
 0002:0000002c       __imp___C_specific_handler 1000302c     corelib1:COREDLL.dll
 0002:00000030       __imp_free                 10003030     corelib1:COREDLL.dll
 0002:00000034       __imp___security_gen_cookie2 10003034     corelib1:COREDLL.dll
 0002:00000038       \177COREDLL_NULL_THUNK_DATA 10003038     coredll:COREDLL.dll
 0002:0000003c       __imp_I2COpenHandle        1000303c     i2csdk:I2CSDK.dll
 0002:00000040       __imp_I2CSetMasterMode     10003040     i2csdk:I2CSDK.dll
 0002:00000044       __imp_I2CSetFrequency      10003044     i2csdk:I2CSDK.dll
 0002:00000048       __imp_I2CTransfer          10003048     i2csdk:I2CSDK.dll
 0002:0000004c       __imp_I2CCloseHandle       1000304c     i2csdk:I2CSDK.dll
 0002:00000050       \177I2CSDK_NULL_THUNK_DATA 10003050     i2csdk:I2CSDK.dll
 0002:00000058       ?dpCurSettings@@3U_DBGPARAM@@A 10003058     DebugZones.obj
 0002:00000524       __security_cookie          10003524     corelib0:seccinit.obj
 0002:00000528       __security_cookie_complement 10003528     corelib0:seccinit.obj
 0002:00000530       _exitflag                  10003530     corelib0:cexit.obj
 0002:00000534       __onexitend                10003534     <common>
 0002:00000538       __onexitbegin              10003538     <common>
 0002:0000053c       g_pcsExit                  1000353c     <common>
 0002:00000540       _pRawDllMain               10003540     <common>

 entry point at        0001:00000d80

 Static symbols

 0001:000003c4       ?ReadI2CRegister@@YAHPAXEEPAEG@Z 100013c4 f   lcdeeprom.obj
 0001:00000440       ?ReadI2CRegister@@YAHPAXEGPAEG@Z 10001440 f   lcdeeprom.obj
 0001:000005a0       ?DetectEEPROM@@YA?AW4EEPROM_TYPE@@PAX@Z 100015a0 f   lcdeeprom.obj
 0001:0000066c       ?IsValidPanelType@@YAHK@Z  1000166c f   lcdeeprom.obj
 0001:000006cc       ?GetPanelType@@YAKPAX@Z    100016cc f   lcdeeprom.obj
 0001:00000784       ?WriteMode@@YAXPAXK@Z      10001784 f   lcdeeprom.obj
 0001:00000888       ?WriteMode32@@YAXPAXK@Z    10001888 f   lcdeeprom.obj
 0001:00000c84       _DllMainCRTStartupHelper   10001c84 f   corelib0:pegdmain.obj
 0001:00000db0       doexit                     10001db0 f   corelib0:cexit.obj
